:1000000015308A003E2D0000FF00030E8301A10081
:100010000A08A0008A010408A2007708A300780853
:10002000A4007908A5007A08A600831383128C30F7
:100030008400001C1D280C1832288B1E21280B1947
:100040003528220884002308F7002408F800250832
:10005000F9002608FA0020088A00210E8300FF0E0E
:100060007F0E09008A110A1223298A110A12912986
:100070008E30F70003174508F8004408F900FA012C
:10008000F808031D4D287908F800F9010830F70237
:10009000F808031D4D28F70155280310F81B5428B4
:1000A000F90DF80DF7034D28F81303130800031793
:1000B000560803191D29E2005A0803191D29E202F6
:1000C000031C67287F30E20703181D296D28813043
:1000D000E202031C1D2903191D296208F700F8011B
:1000E000F901FA01E1015708E000E0175808DF00C4
:1000F0005908DE001930E2005D08DE02031890287E
:100100000130DF0203189028E00203189028E10272
:1001100003189028E10AE00ADF0A5D08DE07C2281A
:100120005C08DF020318AB280130E0020318AB289B
:10013000E1020318AB28E10AE00A5C08DF075D086A
:10014000DE07031CC228DF0A031DC228E00A031DC4
:10015000C228E10AC2285B088038E0020318C128DF
:100160000130E1020318C128E10A5B088038E0078A
:100170005C08DF07031C9F28E00A031D9F28E10A93
:100180009F287A14E20BC528D0280310DE0DDF0D5E
:10019000E00DE10D0310FA0DF90DF80DE30D7C28CB
:1001A000631CD8280310F80CF90CFA0CE30CDB28BC
:1001B000F70303191D29E31B04290310DE0DDF0DCE
:1001C000E00DE10D5D08DE020318F0280130DF02CA
:1001D0000318F028E0020318F028E102031C132999
:1001E0005C08DF020318FB280130E0020318FB283B
:1001F000E102031C13295B088038E002031804297C
:100200000130E102031C1329FA0A031D1329F90A1C
:10021000031D1329F80A031D1329F70A03191D29C1
:10022000F80CF90CFA0C5708E2005B08E206E21F32
:100230001B29F8172129F8132129F701F801F901E1
:10024000FA01031308002C080317B80003132B0846
:100250000317B700BA01FF30B9001030BB00F70137
:10026000FA01B80CB70C031C3B293908F70703182F
:10027000FA0A3A08FA07FA0CF70CF90CF80CBB0B5F
:1002800031297908B8007808B7000313010803176B
:10029000B7070318B80A3808C5003708C4000313A5
:1002A00038207A080317D9007908D8007808D700D1
:1002B0007708D6008030DD00DC01DB017E30DA001B
:1002C000031357207A08B0007908AF007808AE0011
:1002D0007708AD0030080317D90003132F08031760
:1002E000D80003132E080317D70003132D08031794
:1002F000D600DD01DC01DB018030DA00031357207A
:100300007A08B0007908AF007808AE007708AD0031
:10031000AC01AB0181018F018E010C108A110A1210
:100320002128AB0A0319AC0A0B118A110A122128E1
:100330000D050D052310CD32F4326F396F36EF33D2
:10034000E931EB30A039F430EE34E332A01273100F
:10035000A82129103218B119A03BF73BAE36EC307A
:100360006217633DA0060A00301731000D05231007
:10037000C13AF437721DA0127310D037733665324C
:10038000EE34A03A7039613B611DA01273100D0567
:100390000001CA306E104334F237F5397400B11AD7
:1003A0002E1A2E19B01833002310F6327210F037BF
:1003B000F230E434200061346C34743469346D34C8
:1003C000653474345F3474345B34B03443345D3436
:1003D000203461346C34743469346D34653474346D
:1003E0005F3461345B346D345D34203461346C349B
:1003F000743469346D34653474345F3470345B3410
:10040000503461345D3420340034733468347434CF
:100410005F3474345B34B03443345D34203473342B
:10042000683474345F3468345B34253425345D3487
:100430002034203441346E3465346D346F345B3491
:100440006D342F3473345D3463346834653463340D
:100450006B340D340A340D340A3400340830F8009B
:100460000000071228122808831687000000831254
:100470000317920D03138711031C442AA81528089B
:1004800083168700482A8312A8112808831687003C
:100490000000831228162808831687008312071E7F
:1004A0004F2AF80B302A000007122812280883165A
:1004B000870000008312A815280883168700000013
:1004C0000000831228162808831687008312071E4F
:1004D000672AF801000087197814071228122808E3
:1004E0008316870083128711A811280883168700B6
:1004F00083120800A81528088316870000008312BD
:100500002816280883168700000083128711A81177
:100510002808831687000000831207122812280873
:1005200083168700803083120317920003132E2254
:10053000FE300317920003132E22A81128088316F9
:10054000870000008312281628088316870083126C
:10055000071EA82A0000AC2A0000A8152808831648
:100560008700000083128A110A16B02D0830031785
:100570009300770894000313A815280883168700B2
:100580000000831228162808831687008312071E8E
:10059000C72A87190314871D0310F80D00002812BD
:1005A000280883168700831207120317930BBB2AB0
:1005B0000313A815280883168700000083128711EB
:1005C000031714080319EB2A0313A811280883162C
:1005D00087008312031700000313281628088316C8
:1005E00087008312071EF22A00000712281228082B
:1005F00083168700000083128711A811280883162C
:10060000870083120800E230840083130008031976
:10061000162B0230F800F701F70B0C2BF80B0B2B05
:100620009730F700F70B122B800B092B0800A81549
:1006300028088316870000008312281628088316CE
:100640008700000083128711A811280883168700ED
:1006500000008312071228122808831687008030B2
:1006600083120317920003132E22E7300317920020
:1006700003132E22A8152808831687000000831272
:10068000281628088316870000008312071E462BB1
:100690008711A8112808831687000000831207120B
:1006A00028122808831687008130831203179200CE
:1006B00003132E22F701B62278088316DE005E08A7
:1006C0003A395D04DE008312A815280883168700D6
:1006D0000000831228162808831687000000831262
:1006E000071E702B8711A8112808831687000000A9
:1006F000831207122812280883168700803083127D
:100700000317920003132E22E630031792000313FF
:100710002E2283165E0883120317920003132E22E3
:10072000A8112808831687000000831228162808BD
:10073000831687008312071E9B2B00009F2B00004F
:10074000A81528088316870000000A30E2008312EB
:100750000323A81528088316870000008312281693
:10076000280883168700000083128711A811280823
:1007700083168700000083120712281228088316A8
:100780008700803083120317920003132E22E73074
:100790000317920003132E22A8152808831687003A
:1007A0000000831228162808831687000000831291
:1007B000071ED82B8711A811280883168700000070
:1007C00083120712281228088316870081308312AB
:1007D0000317920003132E22F701B622780883161E
:1007E000DE005E08F80083128A110A16B82DA815DB
:1007F000280883168700000083122816280883160D
:100800008700000083128711A8112808831687002B
:1008100000008312071228122808831687003C3034
:1008200083120317920003132E220317920103135E
:100830002E2270300317920003132E22A8112808CD
:100840008316870000008312281628088316870065
:100850008312071E292C00002D2C0000A815280843
:100860008316870000000630E20083120323A815D8
:10087000280883168700000083122816280883168C
:100880008700000083128711A811280883168700AB
:1008900000008312071228122808831687003C30B4
:1008A00083120317920003132E22013003179200C4
:1008B00003132E22E0300317920003132E22A811F7
:1008C000280883168700000083122816280883163C
:1008D00087008312071E6A2C00006E2C0000A815EA
:1008E00028088316870000000630E20083120323E5
:1008F000A8152808831687000000831228162808E8
:1009000083168700000083128711A8112808831618
:100910008700000083120712281228088316870018
:100920003C3083120317920003132E220230031768
:10093000920003132E220317920103132E22A811F3
:1009400028088316870000008312281628088316BB
:1009500087008312071EAA2C0000AE2C0000A815E9
:1009600028088316870000000630E2008312032364
:100970008A110A16C12DA8152808831687000000C1
:100980008312281628088316870000008312871117
:10099000A811280883168700000083120712281266
:1009A000280883168700C0308312031792000313B0
:1009B0002E2226300317920003132E22B83003177D
:1009C000920003132E22A811280883168700000026
:1009D000831228162808831687008312071EEE2C20
:1009E0000000F22C0000A8152808831687000000DC
:1009F0008312A81528088316870000008312281682
:100A0000280883168700000083128711A811280880
:100A10008316870000008312071228122808831605
:100A20008700C03083120317920003132E22133065
:100A30000317920003132E220730031792000313AB
:100A40002E22A8112808831687000000831228167A
:100A50002808831687008312071E2C2D0000302DD6
:100A60000000A81528088316870000008312A81527
:100A7000280883168700000083122816280883168A
:100A80008700000083128711A811280883168700A9
:100A90000000831207122812280883168700C0302E
:100AA00083120317920003132E222630031792009D
:100AB00003132E2239300317920003132E22A8119C
:100AC000280883168700000083122816280883163A
:100AD00087008312071E6A2D00006E2D0000A815E6
:100AE000280883168700000083128A110A16CD2D6C
:100AF000A8152808831687000000831228162808E6
:100B000083168700000083128711A8112808831616
:100B10008700000083120712281228088316870016
:100B2000C03083120317920003132E2203171008FC
:100B3000920003132E22A8152808831687000000B0
:100B40008312281628088316870000008312071EC8
:100B5000A72D8711A811280883168700000083128B
:100B600007122812280883168700C1308312031742
:100B7000920003132E22F701B62278080317910082
:100B80000313A81128088316870000008312281673
:100B90002808831687008312071ECC2D0000D02D55
:100BA0000000A81528088316870000008312031789
:100BB0001108F800031308008030831CE22D03178E
:100BC000A60603130317AB01AC012208AA002608EE
:100BD000AA0621080319D02EA900F7002508031939
:100BE000D92EA9020319752E031C332E2608AF0037
:100BF000AF172708AE002808AD00AC010310AF0CFA
:100C0000AE0CAD0CAC0CA90BFD2DAA1F0A2E2B149B
:100C1000ED2E2B1029102B16243084008317022F61
:100C20002B12AA1B1D2E291C282EAF0CAE0CAD0CAE
:100C3000AC0CF70A0319E82E282EAF1B2B2E03103D
:100C4000AC0DAD0DAE0DAF0DF7030319E82E1D2E43
:100C50002B17952E2B132208AA00AA1F312EAF178F
:100C6000E12EAF13E12E2508A900F7002108A90203
:100C70002208AF00AF172308AE002408AD00AC0176
:100C80000310AF0CAE0CAD0CAC0CA90B3F2EAA1F81
:100C90004C2EAB14ED2EAB102910AB16283084006F
:100CA0008317022FAB12AA1B5F2E291C6A2EAF0CD2
:100CB000AE0CAD0CAC0CF70A0319E82E6A2EAF1B74
:100CC0006D2E0310AC0DAD0DAE0DAF0DF703031976
:100CD000E82E5F2EAB17952EAB132608AA00AA1F8D
:100CE000732EAF17E12EAF13E12E2608AF00AF171A
:100CF0002708AE002808AD00AA1F822EAF132B15BF
:100D0000ED2E2B11AC012910243084008317022F03
:100D1000AA1BAB2E2208AA00291C952EAF0CAE0CE4
:100D2000AD0CAC0CF70A0319E82EAC1FA62EAD0AC9
:100D3000031DA62EAE0A031DA62EAF0A031DA62E66
:100D4000AF0CAE0CAD0CF70A0319E82E2B1B2A2EA4
:100D5000AB1B6C2ECA2E8030AF06AF1FB32EED2E0C
:100D60002608AA00C02E2208AA00AF08031DC02E24
:100D7000AE08031DC02EAD08031DC02EF701E12EE5
:100D8000AF1BCA2E0310AC0DAD0DAE0DAF0DF70BA2
:100D9000C02EE82EAA1FCE2EAF17E12EAF13E12EE4
:100DA0002508F7002608AF002708AE002808AD0088
:100DB000E12E2108F7002208AF002308AE00240826
:100DC000AD002F08F8002E08F9002D08FA00202F9A
:100DD000F701F801F901FA01202FAC01AD09AE09C4
:100DE000AF09AC09AC0A031DFB2EAD0A031DFB2E97
:100DF000AE0A0319AF0A2B18092EAB184B2E2B196C
:100E0000812EB02E0008AD07031C0C2FAE0A031D67
:100E10000C2FAF0A0319291484030008AE07031C22
:100E2000142FAF0A0319291484030008801F803A85
:100E3000AF07031829142B1A102EAB1A522E882E26
:100E40000313080004300317900003137825780873
:100E50008316DD00053083120317900003137825F5
:100E6000780EF7000F30F7057708A7018B1BA7173F
:100E70008B130317C501C40003133820A71B8B175E
:100E800077088316E6007808E7007908E8007A0812
:100E9000E9008312A7018B1BA7178B138316690820
:100EA00083120317D90083160313680883120317EC
:100EB000D80083160313670883120317D70083161D
:100EC0000313660883120317D600DD01DC01DB0182
:100ED0008330DA0003135720A71B8B177A08831679
:100EE000E1007908E0007808DF007708DE0083126F
:100EF000A7018B1BA7178B130317C50183160313B9
:100F00005D0883120317C40003133820A71B8B1737
:100F100083107A080317A4007908A3007808A200B8
:100F20007708A10083160313610883120317A80032
:100F300083160313600883120317A7008316031395
:100F40005F0883120317A600831603135E0883123B
:100F50000317A5000313DC257A088316E50079083A
:100F6000E4007808E3007708E2006208F70063080D
:100F7000F8006408F9006508FA0083128A110A165D
:100F8000DB2D03179401831603136F0883120317D5
:100F90009300940093011008130791001408920025
:100FA0000318920A1108F8001208F9000313080048
:100FB0008E30F70003171108F8001008F900FA0145
:100FC000911FE72FF809F909F90A0319F80AF80837
:100FD000031DF42F7908F800F9010830F702F8082A
:100FE000031DF42FF701FD2F0310F81BFB2FF90D44
:0E0FF000F80DF703F42F911FF81303130800F8
:101000000130031790008A11031378258A1583167F
:10101000E001DF01DE017808DD00023083120317F2
:1010200090008A11031378258A158316E201780847
:10103000E10003308312031790008A11031378250F
:101040008A1578088316E300630DE400E40DFC3094
:10105000E405630EF700F70CF70C0330F70577088B
:101060008312A7018B1BA7178B130317C501C4009D
:101070008A11031338208A15A71B8B1777080317CB
:10108000910078089200790893007A08940003137D
:10109000A7018B1BA7178B1303171408D90013087C
:1010A000D8001208D7001108D600DD01DC01DB01F1
:1010B0008130DA008A11031357208A15A71B8B177A
:1010C0007A088316EC007908EB007808EA007708C4
:1010D000E900831203179101831603135D0D831238
:1010E00003179200831603135E0D831203179300F8
:1010F000831603135F0D831203179400920D930D53
:10110000940DFC30920583160313610DF900620DF6
:10111000FA00F90DFA0DFC30F9057908831203176E
:1011200091047A08920483160313630EF700F70CF8
:10113000F70C0330F7057708831203171104F70043
:101140001208F8001308F9001408FA007A089A0047
:10115000790899007808980077089700B630F7006A
:10116000FA01F901F8011708180419041A04031DFB
:10117000BB28F701C8280310F81BC728970D980D46
:10118000990D9A0DFA0DF90DF80DF70BBB28F81310
:101190007708910078089200790893007A08940003
:1011A00083101408A4001308A3001208A200110859
:1011B000A100831603136C0883120317A80083167B
:1011C00003136B0883120317A700831603136A081F
:1011D00083120317A60083160313690883120317EB
:1011E000A5008A110313DC258A157A088316E80006
:1011F0007908E7007808E6007708E5006508F70059
:101200006608F8006708F9006808FA0083128A1176
:101210000A16E72DA81528088316870000008312F8
:101220002816280883168700000083128711A8114A
:101230002808831687000000831207122812280846
:1012400083168700C0308312031792008A1103139C
:101250002E228A152630031792008A1103132E229C
:101260008A15B830031792008A1103132E228A15AB
:10127000A811280883168700000083122816280862
:10128000831687008312071E4329000047290000A8
:10129000A81528088316870000008312A8152808BF
:1012A00083168700000083122816280883168700FB
:1012B000000083128711A8112808831687000000F8
:1012C000831207122812280883168700C030831261
:1012D000031792008A1103132E228A151330031765
:1012E00092008A1103132E228A15073003179200E9
:1012F0008A1103132E228A15A81128088316870045
:101300000000831228162808831687008312071E00
:10131000872900008B290000A8152808831687005C
:1013200000008312A8152808831687000000831286
:101330002816280883168700000083128711A81139
:101340002808831687000000831207122812280835
:1013500083168700C0308312031792008A1103138B
:101360002E228A152630031792008A1103132E228B
:101370008A15B930031792008A1103132E228A1599
:10138000A811280883168700000083122816280851
:10139000831687008312071ECB290000CF29000087
:1013A000A815280883168700000083128A110A16E0
:1013B000F42D0130031790008A11031378258A1544
:1013C0008316DE017808DD000230831203179000D7
:1013D0008A11031378258A1578088316DF000330F5
:1013E0008312031790008A11031378258A15780E4B
:1013F000F7000F30F7057708A7018B1BA7178B1392
:101400000317C501C4008A11031338208A15A71BCE
:101410008B1777088316E8007808E9007908EA0056
:101420007A08EB008312A7018B1BA7178B13831677
:101430006B0883120317D900831603136A088312FB
:101440000317D80083160313690883120317D70004
:1014500083160313680883120317D600DD01DC012D
:10146000DB018330DA008A11031357208A15A71B8A
:101470008B177A088316E3007908E2007808E10008
:101480007708E0005D08EA00E90169085F04F700F9
:101490005D08FA0077088312A7018B1BA7178B132F
:1014A0000317C4007A08C5008A11031338208A156F
:1014B000A71B8B1777088316E9007808EA007908DC
:1014C000EB007A08EC0083106C0883120317A40069
:1014D000831603136B0883120317A30083160313E9
:1014E0006A0883120317A200831603136908831284
:1014F0000317A10083160313630883120317A800C0
:1015000083160313620883120317A70083160313BD
:10151000610883120317A600831603136008831261
:101520000317A5008A110313DC258A157A08831690
:10153000E7007908E6007808E5007708E400640829
:10154000F7006508F8006608F9006708FA008312DA
:101550008A110A16042E0317210803191C2BA9004F
:10156000250803191C2BA9070318BD2A7F30A902DF
:10157000031C1C2B03191C2BC12A8130A90703183B
:101580001C2B2908F700F801F901FA012208AD0027
:10159000AD172308AC002408AB001830A900AA013D
:1015A0002B1CEA2A2808FA07031CDC2AF90A031D67
:1015B000DC2AF80A0319AA172708F907031CE32AEB
:1015C000F80A0319AA172608A300A3172308F80787
:1015D0000318AA17AA0DF80CF90CFA0CAD0CAC0CF8
:1015E000AB0C0310A90BCF2A0130F70703181C2BF3
:1015F000F81B012BAD0DFA0DF90DF80DF7030319CA
:101600001C2BAD1F122BFA0A031D122BF90A031D06
:10161000122BF80A031D122BF80CF90CFA0CF70A1E
:1016200003191C2B2208AA002608AA06AA1F1A2B97
:10163000F817202BF813202BF701F801F901FA0114
:1016400003130800A81528088316870000008312DA
:10165000281628088316870000008312071E2E2BE9
:101660008711A8112808831687000000831207122B
:1016700028122808831687008030831203179200EF
:101680008A1103132E228A15E330031792008A1160
:1016900003132E228A15A81128088316870000003C
:1016A000831228162808831687008312071E562BDC
:1016B00000005A2B0000A815280883168700000098
:1016C0006430E2008A11831203238A15A8152808C2
:1016D00083168700000083122816280883168700C7
:1016E000000083128711A8112808831687000000C4
:1016F000831207122812280883168700813083126C
:10170000031792008A1103132E228A150130F70065
:101710008A11B6228A1578088316DD000130F70099
:101720008A118312B6228A1578088316DE00F70123
:101730008A118312B6228A1578088316DF00831275
:10174000A81128088316870000008312281628088D
:10175000831687008312071EAB2B0000AF2B0000FF
:10176000A8152808831687000000DE0CDE0C3F3029
:10177000DE05E3015D08E200E300E2015E0EF70032
:10178000F030F70577086207E0006308E10003180E
:10179000E10A8312A7018B1BA7178B13831661081D
:1017A00083120317C50083160313600883120317FF
:1017B000C4008A11031338208A15A71B8B177708DA
:1017C0008316E2007808E3007908E4007A08E5006F
:1017D0008312A7018B1BA7178B138316650883122F
:1017E0000317D90083160313640883120317D80064
:1017F00083160313630883120317D700831603139A
:10180000620883120317D600DD01FF30DC007F3051
:10181000DB008E30DA008A11031357208A15A71BCC
:101820008B1752300317A400B830A3002F30A2004A
:101830008630A1007A08A8007908A7007808A600D9
:101840007708A5000313AB22831066300317A400AA
:10185000A300BB30A2008430A1007A08A800790858
:10186000A7007808A6007708A5008A110313DC25D5
:101870008A158A110A16112EA815280883168700C2
:1018800000008312281628088316870000008312A0
:101890008711A811280883168700000083120712F9
:1018A00028122808831687008030831203179200BD
:1018B0008A1103132E228A15E530031792008A112C
:1018C00003132E228A1564308316E2008A118312D4
:1018D00003238A15A81528088316870000008312A1
:1018E000281628088316870000008312071E762C0E
:1018F0008711A81128088316870000008312071299
:10190000281228088316870081308312031792005B
:101910008A1103132E228A150130F7008A11B6228C
:101920008A1578088316DD000130F7008A118312CA
:10193000B6228A1578088316DE00F7018A11831211
:10194000B6228A1578088316DF008312A8112808AA
:101950008316870000008312281628088316870044
:101960008312071EB12C0000B52C0000A815280812
:10197000831687000000DE0CDE0C3F30DE05E3013D
:101980005D08E200E300E2015E0EF700F030F705CB
:1019900077086207E0006308E1000318E10A831298
:1019A000A7018B1BA7178B138316610883120317DC
:1019B000C50083160313600883120317C4008A113D
:1019C000031338208A15A71B8B1777088316E200AC
:1019D0007808E3007908E4007A08E5008312A7019B
:1019E0008B1BA7178B138316650883120317D90067
:1019F00083160313640883120317D8008316031396
:101A0000630883120317D700831603136208831237
:101A10000317D600DD01FF30DC007F30DB008E30A5
:101A2000DA008A11031357208A15A71B8B17031797
:101A3000A401A3017A30A2008530A1007A08A80091
:101A40007908A7007808A6007708A5000313AB2241
:101A500083100317A401A301C030A2008130A100AC
:101A60007A08A8007908A7007808A6007708A500DA
:101A70008A110313DC258A158A110A161E2EA81551
:101A8000280883168700000083122816280883166A
:101A90008700000083128711A81128088316870089
:101AA00000008312071228122808831687003C3092
:101AB0008312031792008A1103132E228A158316AC
:101AC0006F088312031792008A1103132E228A15BE
:101AD000A8112808831687000000831228162808FA
:101AE000831687008312071E732D0000772D0000D8
:101AF000A81528088316870000008312A815280857
:101B00008316870000008312281628088316870092
:101B1000000083128711A81128088316870000008F
:101B20008312071228122808831687003D3083127B
:101B3000031792008A1103132E228A15F7018A11C6
:101B4000B6228A1578088316EF006F08F800831212
:101B5000080003171E08A5002208A506A51FB52D1D
:101B6000031103109E1B0314E82D1E08A500210875
:101B7000A6001D08A6020319C32DA51FE82D030802
:101B8000013A8300E82D2208A6001E08A6020319C8
:101B9000CF2DA51FE82D0308013A8300E82D230867
:101BA000A6001F08A6020319DB2DA51FE82D0308B8
:101BB000013A8300E82D2408A6002008A602031994
:101BC000E72DA51FE82D0308013A8300E82D031037
:101BD0000313080031088400831332188317831617
:101BE0006A088000840A80018312B10A0319B20ACC
:101BF0000800F701F801F901FA01031794019501B2
:101C000096019701130812041104100403193C2EC5
:101C100020309800031083160313EA0DEB0DEC0D32
:101C2000ED0D83120317940D950D960D970D130866
:101C30001702031D252E12081602031D252E11085A
:101C40001502031D252E10081402031C362E100841
:101C500094021108031C110F95021208031C120FA5
:101C600096021308031C130F97020314F70DF80DC7
:101C7000F90DFA0D980B0A2E143084008317031304
:101C8000080004088316E2006108E4000319712EBD
:101C9000600883120317A400831603135F088312DE
:101CA0000317A300831603135E0883120317A20011
:101CB000831603135D0883120317A100A801A7016F
:101CC0002030A6008230A5000313AB227A088316C9
:101CD000E0007908DF007808DE007708DD00E40B1B
:101CE000482E6008ED005F08EC005E08EB005D0820
:101CF000EA006A08B63CEA00FA016B08EE00EB174E
:101D00000310EB0CEC0CED0CFA0CF90CF80CF70CC6
:101D1000EA0B802EEE1F972EF709F809F909FA0948
:101D2000F70A0319F80A0319F90A0319FA0A7A08D3
:101D3000E0007908DF007808DE007708DD00E01FAA
:101D4000AE2EE203E216DD09DE09DF09E009DD0A55
:101D50000319DE0A0319DF0A0319E00A3B30E90020
:101D60009A30E800CA30E700E6010A30E400610872
:101D70000319E20A6008ED005F08EC005E08EB0062
:101D80005D08EA00690883120317930083160313A2
:101D900068088312031792008316031367088312DF
:101DA000031791008316031366088312031790002C
:101DB0000313F92500088316DD00840A0008DE00FD
:101DC000840A0008DF00840A0008E000FD30840770
:101DD000F708031DFE2E610A64020319FE2E620835
:101DE0000319002F0F3964020319F82E0318382F36
:101DF000E21B382F621B002F2030322F2030E205EB
:101E0000E21E102FE2126108031DE2037708E200D0
:101E10002D30EA008312EA2583166208F700E201FA
:101E200061086402031D202F7708E2002E30EA00CB
:101E30008312EA2583166208F7002030E20500309D
:101E40003030E21E322FE2126108031DE2037708F0
:101E5000E2002D30EA008312EA2583166208F700BB
:101E6000E2013030F7077708EA008312EA2583168B
:101E70006908ED006808EC006708EB006608EA00F6
:101E8000831203179301920191010A30900003130A
:101E9000F9257A088316E9007908E8007808E70050
:101EA0007708E600E40BBA2E8312080080080319B5
:101EB000962F8316DE010408DD005E10831B5E147E
:101EC0000008DF008312A8132808831687008312F6
:101ED00087130830F8006C2F0000F8177F2FF813D5
:101EE0008316DF0C831203188717031C87137817D8
:101EF0007F2F7813F80B702F7D2F000087173F304E
:101F00008400840B812F0000F81B6F2F781B792F22
:101F100083165D08840083135E188317840A031DEB
:101F2000942F8312850A83168312562F8A110A165C
:021F3000282F58
:1020000003308316EF000A128A1583123F250A1641
:102010008A1178088316EB000430EF000A128A1543
:1020200083123F250A168A1178088316EC006B0884
:10203000EF006C088312031790000A120313C127E4
:102040000A1679088316EE007808ED006D08F8008E
:102050006E08F9007908DE007808DD000730EF002F
:102060000A128A1583123F250A168A1178088316E8
:10207000EB000830EF000A128A1583123F250A167A
:102080008A1178088316EC006B08EF006C08831245
:10209000031790000A120313C1270A167908831642
:1020A000EE007808ED006D08F8006E08F900790878
:1020B000E0007808DF000530EF000A128A1583126D
:1020C0003F250A168A1178088316EB000630EF00C8
:1020D0000A128A1583123F250A168A117808831678
:1020E000EC006B08EF006C088312031790000A12D3
:1020F0000313C1270A1679088316EE007808ED004D
:102100006D08F8006E08F9007908E2007808E1002F
:102110006008831203179100831603135F0883126C
:10212000031790000A120313D8270A16770883169C
:10213000EB007808EC007908ED007A08EE005E0804
:10214000831203179100831603135D08831203178C
:1021500090000A120313D8270A16A7018B1BA71792
:102160008B1383166E0883120317D900831603138B
:102170006D0883120317D800831603136C088312AB
:102180000317D700831603136B0883120317D600B7
:102190007A08DD007908DC007808DB007708DA00CF
:1021A0000A12031357200A16A71B8B177A088316E7
:1021B000E6007908E5007808E4007708E30066089F
:1021C000EE006508ED006408EC006308EB006F109A
:1021D000EF106E08831203179300831603136D0824
:1021E000831203179200831603136C0883120317DC
:1021F0009100831603136B08831203179000831654
:1022000003136E0883120317A000831603136D08CF
:10221000831203179F00831603136C08831203179E
:102220009E00831603136B08831203179D00A401FD
:10223000A301A201A1010A128A150313A9250A16F6
:102240008A11031C2B2983166F148312031711089C
:10225000803A910003130317A0019F019E017F3074
:102260009D001308A4001208A3001108A200100882
:10227000A1000A128A150313A9250A168A11031C44
:102280006629A7018B1BA7178B130317D901D80148
:10229000D7017F30D6001308DD001208DC001108DA
:1022A000DB001008DA000A12031357200A16A71BD6
:1022B0008B177A0803179300790892007808910029
:1022C0007708900083160313EF1483120A30031764
:1022D000A4008930A3003430A2007C30A100130890
:1022E000A8001208A7001108A6001008A5000A12ED
:1022F0008A150313AB220A168A11770803179C006C
:1023000078089D0079089E007A089F00A4001E08A6
:10231000A3001D08A2001C08A1001308A8001208B1
:10232000A7001108A6001008A5000A128A150313B9
:10233000AB220A168A11770803179C0078089D00C3
:1023400079089E007A089F0083101F08A4001E08C9
:10235000A3001D08A2001C08A1007C30A800793051
:10236000A7003530A6008130A5000A120313DC2532
:102370000A167A08031797007908960078089500DE
:10238000770894001708A4001608A3001508A200F7
:102390001408A1001308A8001208A7001108A6003D
:1023A0001008A5000A128A150313AB220A168A1117
:1023B000770803179C0078089D0079089E007A082A
:1023C0009F00A4001E08A3001D08A2001C08A10075
:1023D0001308A8001208A7001108A6001008A500FD
:1023E0000A128A150313AB220A168A1177080317FB
:1023F0009C0078089D0079089E007A089F00831051
:102400001F08A4001E08A3001D08A2001C08A100AC
:102410003F30A8000230A7003330A6008330A5006B
:102420000A120313DC250A167A08031797007908A5
:10243000960078089500770894001708A4001608FD
:10244000A3001508A2001408A1001308A800120890
:10245000A7001108A6001008A5000A128A15031388
:10246000AB220A168A11770803179C0078089D0092
:1024700079089E007A089F00A4001E08A3001D088A
:10248000A2001C08A1001308A8001208A700110848
:10249000A6001008A5000A128A150313AB220A161B
:1024A0008A11770803179C0078089D0079089E0020
:1024B0007A089F0083101F08A4001E08A3001D08AF
:1024C000A2001C08A1003330A8008C30A7001E30E9
:1024D000A6008330A5000A120313DC250A167A0829
:1024E00003179700790896007808950077089400FC
:1024F000A401A301A2017F30A1001308A8001208C3
:10250000A7001108A6001008A5000A128A150313D7
:10251000AB220A168A11770803179C0078089D00E1
:1025200079089E007A089F00A4001E08A3001D08D9
:10253000A2001C08A1001308A8001208A700110897
:10254000A6001008A5000A128A150313AB220A166A
:102550008A11770803179C0078089D0079089E006F
:102560007A089F0083101F08A4001E08A3001D08FE
:10257000A2001C08A1001B30A800E430A7003530E1
:10258000A6008230A5000A120313DC250A167A0879
:1025900003179B0079089A0078089900770898003B
:1025A0001B08A4001A08A3001908A2001808A1001B
:1025B0001308A8001208A7001108A6001008A5001B
:1025C0000A128A150313AB220A168A117708031719
:1025D0009C0078089D0079089E007A089F00A4005E
:1025E0001E08A3001D08A2001C08A1001308A800D3
:1025F0001208A7001108A6001008A5000A128A15E3
:102600000313AB220A168A11770803179C00780877
:102610009D0079089E007A089F0083101F08A4007F
:102620001E08A3001D08A2001C08A100A430A800D9
:10263000DB30A7006730A6008330A5000A12031321
:10264000DC250A167A0803179B0079089A00780897
:102650009900770898001B08A4001A08A30019081D
:10266000A2001808A1001308A8001208A70011086A
:10267000A6001008A5000A128A150313AB220A1639
:102680008A11770803179C0078089D0079089E003E
:102690007A089F00A4001E08A3001D08A2001C08C1
:1026A000A1001308A8001208A7001108A60010082E
:1026B000A5000A128A150313AB220A168A1177089D
:1026C00003179C0078089D0079089E007A089F00F7
:1026D00083101F08A4001E08A3001D08A2001C08E8
:1026E000A1003330A8008C30A7001E30A600833034
:1026F000A5000A120313DC250A167A0803179B00AB
:1027000079089A0078089900770898001308A400BF
:102710001208A3001108A2001008A1001708A800C1
:102720001608A7001508A6001408A5000A128A15A5
:102730000313AB220A168A11770803179C00780846
:102740009D0079089E007A089F000313A7018B1B48
:10275000A7178B1303171F08D9001E08D8001D08E0
:10276000D7001C08D6001B08DD001A08DC00190879
:10277000DB001808DA000A12031357200A16A71BF9
:102780008B177A0803179700790896007808950048
:102790007708940083160313EF1CF02B8314DB30AF
:1027A00083120317A4000F30A3004930A2007F302A
:1027B000A1001708A8001608A7001508A60014080D
:1027C000A5000A120313DC250A167A0803179700DE
:1027D000790896007808950077089400831603130B
:1027E0006F1CF92B831203171508803A9500831686
:1027F0000313831203171408F7001508F8001608CE
:10280000F9001708FA007A0883160313EA0079081A
:10281000E9007808E8007708E7008312A7018B1B1E
:10282000A7178B1383166A0883120317D900831620
:102830000313690883120317D8008316031368086B
:1028400083120317D7008316031367088312031735
:10285000D600C330DD00F530DC004830DB008030CE
:10286000DA000A12031357200A16A71B8B177708E2
:102870008316EB007808EC007908ED007A08EE008A
:1028800083120317A400831603136D088312031722
:10289000A300831603136C0883120317A200831688
:1028A00003136B0883120317A100A801A70134309A
:1028B000A6008630A5000A128A150313AB220A1659
:1028C0008A117A088316EA007908E9007808E80096
:1028D0007708E7006708F7006808F8006908F9005A
:1028E0006A08FA00F8136A08EA006908E90078083B
:1028F000E8006708E700DD08031D982CDE08031DCB
:10290000982CE01B912CE008031D8A2C5F08003CEA
:102910000318912CEA01E9013430E8008530E70022
:10292000972CEA01E9010730E8008730E700322DF3
:10293000DE1B012DDE08031DA12C5D08003C0318E1
:10294000012DE01BD22C831083120317A401A301D5
:102950003430A2008630A100831603136A08831264
:102960000317A80083160313690883120317A7002F
:1029700083160313680883120317A6008316031334
:10298000670883120317A5000A120313DC250A1631
:102990007A088316EA007908E9007808E8007708E1
:1029A000E700002D831483120317A401A301343020
:1029B000A2008630A100831603136A08831203174E
:1029C000A80083160313690883120317A700831650
:1029D0000313680883120317A600831603136708FE
:1029E00083120317A5000A120313DC250A167A08BE
:1029F0008316EA007908E9007808E8007708E7001C
:102A0000322DE01B322D831483120317A401A3017E
:102A10003430A2008730A100831603136A088312A2
:102A20000317A80083160313690883120317A7006E
:102A300083160313680883120317A6008316031373
:102A4000670883120317A5000A120313DC250A1670
:102A50007A088316EA007908E9007808E800770820
:102A6000E700322D6708F7006808F8006908F900E8
:102A70006A08FA0083128A110A16292E8401831328
:102A80001F308305713083168F000F088312A8133F
:102A900028088316870083128717B001AF01AE01A3
:102AA000AD01831603170908C039890003131F12EB
:102AB0009F12003003178800831287018801890163
:102AC000FF300313A800A901AA01B101B2018316C6
:102AD00003170908C039890003131F129F12003021
:102AE00003178800831203131F139F1383169F136A
:102AF00083121F149412A8122808831687008312C9
:102B000028162808831687008312A8112808831620
:102B1000870001308312940000308316940001086E
:102B2000C739283881000F30831290000030F80038
:102B3000920000308316920083122815280883160D
:102B400087008312970183169B019C0101309D0031
:102B5000831203178701880189010A1203137A2A55
:102B60000A16CB014B088316DD000A128312172BBD
:102B70000A1683160C1483128B16C0308B040A12AB
:102B8000F72B0A1681018F018E01AC01AB01B00158
:102B9000AF01AE01AD010A12BB2C0A160230CD0006
:102BA000FA308316E2000A12831203230A16CD0BB1
:102BB000D02D0A12222F0A167A08B6007908B5001D
:102BC0007808B4007708B3000A128A1500280A169C
:102BD0008A117A08BA007908B9007808B80077082D
:102BE000B7000A128A150A290A168A110230CD0086
:102BF000FA308316E2000A12831203230A16CD0B61
:102C0000F82D0A128A15D9290A168A117A08BE00E7
:102C10007908BD007808BC007708BB000A128A1545
:102C2000222B0A168A117A08C2007908C100780896
:102C3000C0007708BF000A128A153C2C0A168A11B8
:102C40007A08C6007908C5007808C4007708C30070
:102C500000287A08CA007908C9007808C8007708EF
:102C6000C700B201A030B10020308316EA000A127A
:102C70008A158312EA250A168A110530840036085F
:102C80008316E000831235088316DF0083123408B0
:102C90008316DE00831233088316DD000230E10064
:102CA0000A128A15831241260A168A1120308316C9
:102CB000EA000A128A158312EA250A168A110630DA
:102CC00084003E088316E00083123D088316DF006F
:102CD00083123C088316DE0083123B088316DD0056
:102CE0000230E1000A128A15831241260A168A115F
:102CF00020308316EA000A128A158312EA250A1682
:102D00008A11083084003A088316E00083123908DB
:102D10008316DF00831238088316DE00831237081B
:102D20008316DD000230E1000A128A158312412663
:102D30000A168A1120308316EA000A128A158312B5
:102D4000EA250A168A110530840042088316E0003D
:102D5000831241088316DF00831240088316DE00C9
:102D600083123F088316DD000230E1000A128A1543
:102D7000831241260A168A1120308316EA000A12AD
:102D80008A158312EA250A168A110530840046083E
:102D90008316E000831245088316DF00831244087F
:102DA0008316DE00831243088316DD000230E10043
:102DB0000A128A15831241260A168A1120308316B8
:102DC000EA000A128A158312EA250A168A110430CB
:102DD00084004A088316E000831249088316DF0046
:102DE000831248088316DE00831247088316DD002D
:102DF0000230E1000A128A15831241260A168A114E
:102E000020308316EA000A128A158312EA250A1670
:102E10008A110530840030088316E00083122F08E1
:102E20008316DF0083122E088316DE0083122D081E
:102E30008316DD000230E1000A128A158312412652
:102E40000A168A11A030840083130A128A15562F9D
:102E50000A168A11CC01CC014C08273C031C3D2FDB
:102E60000430CD00FA308316E2000A1283120323E5
:0E2E70000A16CD0B322FCC0A2C2FCB2D63006F
:04400E00F52CFF3F4F
:00000001FF
